:100000000C9472000C949A000C949A000C949A0030
:100010000C949A000C949A000C949A000C942B0661
:100020000C949A000C949A000C949A000C940D086D
:100030000C949A000C949A000C949A000C949A00D8
:100040000C9475090C949A000C94AD060C948706D8
:100050000C949A000C949A000C949A000C949A00B8
:100060000C94DF060C949A00B10CEA0FEA0F8A0E8A
:10007000B90CEA0FEA0FEA0F200F440F6A0F6A0F5C
:100080006A0FCE0F020000000023002600290000A6
:10009000000000240027002A0000000008000201E0
:1000A000000003040700000000000000000102043B
:1000B00008102040800102040810200102040810EA
:1000C0002000000000250028002B00040404040484
:1000D00004040402020202020203030303030300F6
:1000E0001E121E1311241FBECFEFD8E0DEBFCDBFFE
:1000F00011E0A0E0B1E0E6E4FDE202C005900D925F
:10010000AE35B107D9F723E0AEE5B1E001C01D92ED
:10011000A039B207E1F710E0C1E7D0E004C02197B1
:10012000FE010E946315C037D107C9F70E94040A77
:100130000C9496160C940000682F85ED92E00C94B8
:10014000CB050F931F93CF93DF93CDB7DEB72997DE
:100150000FB6F894DEBF0FBECDBF80910F03909114
:100160001003892B09F4A2C00E94500900911503C5
:10017000109116032091170330911803DC01CB0175
:10018000801B910BA20BB30B8C329140A105B105E2
:1001900058F3F89480910A0390910B039A83898312
:1001A000E0910F03F0911003DF01119680818987A0
:1001B00090910603E0911903F0911A0380911B03BB
:1001C000992309F42EC09081982B9887908180956F
:1001D00089238F838F818C8388E08B8358856F81FF
:1001E00049853B812C8189819A81508347FD252F48
:1001F0003A952083262F39F0441F00C00000608309
:10020000000000C0F2CF38E04D91608300000197FC
:1002100061F7F0931A03E093190349873B832C831A
:1002200038C09081982B98879081809589238F83FF
:100230008F818E8388E08D8358856F8149853D81CC
:100240002E8189819A81508347FD252F00C000C0EF
:10025000208300C000C000C000C000C06083000058
:10026000262F3A9541F0441F000000C000C000C096
:1002700000C000C0E8CF38E04D9100C0608300C0EE
:10028000019709F7F0931A03E093190349873D8317
:100290002E839A83898378940E9450096093150372
:1002A00070931603809317039093180329960FB643
:1002B000F894DEBF0FBECDBFDF91CF911F910F919C
:1002C00008951F93CF93DF9311E0180F20910E0331
:1002D0001217A1F1C0910F03D09110032150B9F072
:1002E0008F3F59F430E040E050E06FEF7FEF80E067
:1002F00090E00E942E13B9010CC0812F90E0982F3E
:1003000088270197622F70E00E944F1502C060E0BD
:1003100070E0FE0140910A0350910B03CF018C1B4A
:100320009D0B8417950740F44081469FC001479F6D
:10033000900D11249193EECF10930E03DF91CF9186
:100340001F91089530913402313208F04BC08091F2
:1003500033028111FCCF90913B0322E020933302C2
:1003600021E0209332022FEF20930B0210920A0219
:1003700030930902EDE0F2E0A9EEB1E020E032179F
:1003800021F041914D932F5FFACF1092E801209117
:10039000E801990F922B9093E801909131029130EE
:1003A00061F4109231029091E8019093BB0090911A
:1003B000BC0093FDF8CF95EC01C095EE9093BC0086
:1003C000909133029230E1F390910B029F3F79F0CC
:1003D00080910B02803241F080910B02803331F02A
:1003E00084E005C081E003C082E001C083E0109298
:1003F00035021092340210920C02089591E090930D
:100400000C0280933B03109235021092340208953F
:100410000F931F93CF93DF93809121030E94FE01DE
:1004200080E090E00E949C000DE113E0C0E0D0E08D
:10043000F80161918F0185ED92E00E94CB058FEF6D
:1004400090E00E949C00C130D10541F480E090E032
:100450000E949C0080E090E00E949C002196C430A5
:10046000D10531F7DF91CF911F910F910C94A2012B
:100470002091080330910903232B81F190910E0301
:10048000992361F0899F90011124832F969FB001D9
:100490001124672F949FA0011124452F90911403DC
:1004A0005091110320910F0330911003951721F003
:1004B000F901E90FF11D108290911103F901E90F83
:1004C000F11D808380911203F901E80FF11D608313
:1004D00080911303F901E80FF11D40830895909175
:1004E00033029111FCCF91E090933302909332024A
:1004F0002FEF20930B0210920A02260F209309027D
:100500009093E8019091E801880F892B8093E8018E
:1005100080913102813061F4109231028091E801C2
:100520008093BB008091BC0083FDF8CF85EC01C0B7
:1005300085EE8093BC00809133028130E1F380919D
:100540000A02861710F460910A02A9EEB1E0E8EC05
:10055000F1E080E0861721F09D9191938F5FFACFB3
:100560000895833081F028F4813099F08230A1F031
:1005700008958730A9F08830B9F08430D1F48091A3
:1005800080008F7D03C0809180008F7780938000F2
:10059000089584B58F7702C084B58F7D84BD08959A
:1005A0008091B0008F7703C08091B0008F7D8093E1
:1005B000B00008951F93CF93DF93282F30E0F90107
:1005C000E756FF4F8491F901E355FF4FD491F901AC
:1005D000E553FF4FC491CC23C1F0162F81110E9427
:1005E000B102EC2FF0E0EE0FFF1FEF53FF4FA5918C
:1005F000B4919FB7F894111104C08C91D095D82371
:1006000002C0EC91DE2BDC939FBFDF91CF911F9155
:10061000089510923702109236021092350210920D
:1006200034021092330281E0809332021092310240
:1006300061E082E10E94DA0261E083E10E94DA0275
:10064000E9EBF0E080818E7F808380818D7F8083E5
:1006500088E48093B80085E48093BC0080E795E04F
:100660009093300280932F0281E795E090932E02C1
:1006700080932D0208951F93CF93DF93CDE1D3E0B4
:100680001C810E940903110F1093BA008C810E94F3
:10069000FE0161E285ED92E00E94CB050E94A2017D
:1006A0008C810E94FE0161E885ED92E00E94CB05FD
:1006B000DF91CF911F910C94A201CF93DF9390E033
:1006C000FC01E355FF4F2491FC01E553FF4F84915A
:1006D000882361F190E0880F991FFC01E157FF4FDB
:1006E000C591D491FC01EF53FF4FA591B4916111D5
:1006F00009C09FB7F8948881209582238883EC9164
:100700002E230BC0623061F49FB7F8948881322F9A
:10071000309583238883EC912E2B2C939FBF06C0AA
:100720008FB7F894E8812E2B28838FBFDF91CF916C
:1007300008951F93CF93DF93182FEB0161E00E9480
:100740005D03209711F460E004C0CF3FD10539F478
:1007500061E0812FDF91CF911F910C94DA02E12F9C
:10076000F0E0E756FF4FE491E330F9F048F4E13070
:10077000B9F0E230A1F584B5806284BDC8BD34C053
:10078000E730E9F0E83019F1E43049F58091800074
:10079000806280938000D0938B00C0938A0024C035
:1007A00084B5806884BDC7BD1FC08091800080680B
:1007B00080938000D0938900C093880015C08091F9
:1007C000B00080688093B000C093B3000DC08091EA
:1007D000B00080628093B000C093B40005C0C03800
:1007E000D1050CF0B5CFAFCFDF91CF911F91089518
:1007F0008F929F92AF92BF92CF92DF92EF92FF9231
:100800006B017C010E9450094B015C01C114D104B1
:10081000E104F104F1F00E945009DC01CB018819D8
:100820009909AA09BB09883E9340A105B10570F357
:1008300021E0C21AD108E108F10888EE880E83E0B1
:10084000981EA11CB11CC114D104E104F10419F7D4
:10085000DDCFFF90EF90DF90CF90BF90AF909F9053
:100860008F900895CF92DF92EF92FF920F931F9394
:10087000CF93DF936C017A018B01C0E0D0E0CE15FD
:10088000DF0581F0D8016D918D01D601ED91FC91CC
:100890000190F081E02DC6010995892B11F0219678
:1008A000EECF7E01C701DF91CF911F910F91FF9095
:1008B000EF90DF90CF900895FC01538D448D252F4C
:1008C00030E0842F90E0821B930B541710F0CF96EA
:1008D000089501970895FC01918D828D981761F01C
:1008E000828DDF01A80FB11D5D968C91928D9F5F67
:1008F0009F73928F90E008958FEF9FEF0895FC0112
:10090000918D828D981731F0828DE80FF11D858DC4
:1009100090E008958FEF9FEF0895FC01918D228D57
:10092000892F90E0805C9F4F821B91098F739927DC
:10093000089588E392E00E948D0421E0892B09F458
:1009400020E0822F0895FC01848DDF01A80FB11DE6
:10095000A35ABF4F2C91848D90E001968F739927F5
:10096000848FA689B7892C93A089B1898C918370D3
:1009700080648C93938D848D981306C00288F389CC
:10098000E02D80818F7D80830895EF92FF920F93F9
:100990001F93CF93DF93EC0181E0888F9B8D8C8D2B
:1009A000981305C0E889F989808185FD26C0F62E57
:1009B0000B8D10E00F5F1F4F0F731127E02E8C8DF2
:1009C000E8120CC00FB607FCFACFE889F9898081DC
:1009D00085FFF5CFCE010E94A304F1CF8B8DFE01E0
:1009E000E80FF11DE35AFF4FF0829FB7F8940B8F89
:1009F000EA89FB89808180620AC09FB7F894EE89FA
:100A0000FF896083E889F9898081837080648083AD
:100A10009FBF81E090E0DF91CF911F910F91FF90F8
:100A2000EF900895CF93DF93EC01888D8823C9F070
:100A3000EA89FB89808185FD05C0A889B9898C91E7
:100A400086FD0FC00FB607FCF5CF808185FFF2CF82
:100A5000A889B9898C9185FFEDCFCE010E94A304AE
:100A6000E7CFDF91CF91089580E090E0892B29F0C6
:100A70000E94990481110C940000089585ED8093E3
:100A8000BC008091BC0084FDFCCF1092330208951D
:100A900040916003262F30E0240F311D21323105B3
:100AA000DCF4209133022430C9F4FC0180E090E0B2
:100AB000861758F4309160032191DC01A05CBC4F93
:100AC000A30FB11D2C930196F3CF80916003680FA3
:100AD0006093600380E0089581E0089582E00895C6
:100AE000089508950895E091370280913602E8173D
:100AF00030F4F0E0E853FE4F808190E008958FEFEE
:100B00009FEF08959091370280913602981750F424
:100B1000E92FF0E0E853FE4F208130E09F5F909393
:100B2000370202C02FEF3FEFC901089580913602CE
:100B300090E020913702821B91090895CF92DF92B5
:100B4000EF92FF920F931F93CF93DF937C01CB0122
:100B50008A0120910C02222389F0EB016B01C40E63
:100B6000D51ECC15DD0569F06991D701ED91FC9199
:100B70000190F081E02DC7010995F3CF642F0E9409
:100B80004805C801DF91CF911F910F91FF90EF9021
:100B9000DF90CF900895CF93DF931F92CDB7DEB74C
:100BA000698320910C022223D1F02091340220325B
:100BB00040F021E030E0FC013383228380E090E0CC
:100BC00015C080913502E82FF0E0E35FFD4F998179
:100BD00090838F5F809335028093340205C061E07B
:100BE000CE0101960E94480581E090E00F90DF91D0
:100BF000CF910895089580E090E008950E949116A5
:100C000090910001891324C0E4E8F0E0E4919FEFA3
:100C100090930001E130B9F098F0E230C9F490917E
:100C200070009D7F9093700091E09093B000909140
:100C3000B100987F94609093B1001092B30008C007
:100C400010926E0005C090916F009D7F90936F0091
:100C500060E00C94DA021F920F920FB60F921124EB
:100C60002F933F934F935F936F937F938F939F93B4
:100C7000AF93BF93EF93FF938091610190916201D5
:100C8000A0916301B0916401892B8A2B8B2B51F1C8
:100C900090915E01E0915F01F09160018081892770
:100CA00080838091610190916201A0916301B09174
:100CB0006401181619061A061B06C4F48091610116
:100CC00090916201A0916301B09164010197A10923
:100CD000B1098093610190936201A0936301B09385
:100CE000640104C0809100010E940006FF91EF9111
:100CF000BF91AF919F918F917F916F915F914F9134
:100D00003F912F910F900FBE0F901F9018951F923B
:100D10000F920FB60F9211242F933F934F935F932F
:100D20006F937F938F939F93AF93BF93EF93FF93B3
:100D300088E392E00E94A304FF91EF91BF91AF91ED
:100D40009F918F917F916F915F914F913F912F91E3
:100D50000F900FBE0F901F9018951F920F920FB615
:100D60000F9211242F938F939F93EF93FF93E09112
:100D70004802F09149028081E0914E02F0914F02C9
:100D800082FD12C09081809151028F5F8F732091FC
:100D90005202821751F0E0915102F0E0E85CFD4F01
:100DA000958F8093510201C08081FF91EF919F91B7
:100DB0008F912F910F900FBE0F901F9018951F923B
:100DC0000F920FB60F9211242F933F934F935F937F
:100DD0006F937F938F939F93AF93BF93EF93FF9303
:100DE0008091B900887F803609F49CC068F588320C
:100DF00009F45BC090F4803109F454C038F48823BE
:100E000009F4F6C0883009F44DC0F6C0883109F401
:100E10004CC0803209F45DC0EFC0803409F468C072
:100E200048F4803309F455C0883309F0E5C0809355
:100E30000B02D8C0803509F44FC0883509F45DC075
:100E4000883409F0D9C0D6C0883909F4C7C0A8F4DD
:100E5000883709F467C038F4883609F463C08037EE
:100E600009F460C0C9C0883809F4B8C0803909F4F1
:100E70005FC0803809F0C0C05BC0803B09F486C009
:100E800038F4803A09F466C0883A09F47FC0B4C0E7
:100E9000803C09F4A7C0883C09F4A4C0883B09F44D
:100EA0008AC0AAC08091E80110C090910A02809186
:100EB0000902981770F5E0910A0281E08E0F809385
:100EC0000A02F0E0E751FE4F80818093BB0085EC81
:100ED00086C080930B028EC0E0910A0281E08E0FE3
:100EE00080930A028091BB00F0E0E751FE4F8083BF
:100EF00090910A02809109026EC0E0910A0281E09D
:100F00008E0F80930A028091BB00F0E0E751FE4F04
:100F100080838091320281116DC081E08093310223
:100F200084EA61C083E08093330210928203CFCFC2
:100F300080918203803208F051C0E091820381E009
:100F40008E0F809382038091BB00F0E0EE59FC4F3E
:100F50008083BDCF85EC8093BC00109233028091DA
:100F60008203803230F4E0918203F0E0EE59FC4FCE
:100F700010826091820370E0E0912D02F0912E02C8
:100F800082E693E009951092820336C084E0809354
:100F900033021092610310926003E0912F02F091EE
:100FA0003002099580916003811105C081E0809332
:100FB000600310924003E091610381E08E0F809303
:100FC0006103F0E0E05CFC4F80818093BB00909176
:100FD000610380916003981708F479CF85E88093C6
:100FE000BC000AC085EC8093BC001092330204C0A0
:100FF00010920B020E943E05FF91EF91BF91AF91BD
:101000009F918F917F916F915F914F913F912F9120
:101010000F900FBE0F901F9018951F920F920FB652
:101020000F9211242F933F934F935F936F937F936E
:101030008F939F93AF93BF93EF93FF9380913F0361
:1010400087FF05C010928500109284001BC020917C
:101050003F03022E000C330B8091050390E028170C
:10106000390784F480913F03082E000C990BFC0192
:10107000EE0FFF1F8E0F9F1FFC01EF51FD4F808170
:1010800086FD15C080913F038F5F80933F032091C1
:101090003F03022E000C330B8091050390E02817CC
:1010A0003907C4F480913F038C3064F113C0809100
:1010B0003F03082E000C990BFC01EE0FFF1F8E0F53
:1010C0009F1FFC01EF51FD4F808160E08F730E94F4
:1010D000DA02D8CF80918400909185000496803404
:1010E0009C4918F480E49CE905C0809184009091AB
:1010F0008500049690938900809388008FEF8093F9
:101100003F033BC0209184003091850080913F03D4
:10111000082E000C990BFC01EE0FFF1F8E0F9F1F76
:10112000FC01EF51FD4F81819281820F931F9093BB
:1011300089008093880080913F03082E000C990B52
:10114000FC01EE0FFF1F8E0F9F1FFC01EF51FD4FA3
:10115000808186FF12C080913F03082E000C990BFE
:10116000FC01EE0FFF1F8E0F9F1FFC01EF51FD4F83
:10117000808161E08F730E94DA02FF91EF91BF914D
:10118000AF919F918F917F916F915F914F913F911F
:101190002F910F900FBE0F901F901895682F88E326
:1011A00092E00C94C504EF92FF920F931F93CF939C
:1011B000DF93162FE72EF82E092F82E00E94CE082B
:1011C000C5E6D1E0812F9E2DAF2DB02F8883998366
:1011D000AA83BB830E94CE0889810E94CE088A819F
:1011E0000E94CE088B81DF91CF911F910F91FF90CC
:1011F000EF900C94CE0842E050E06AE571E088E39D
:1012000092E00C9432048FEF0E94CE0885E50E9494
:10121000CE080C94FB088FEF0E94CE0885E50C9455
:10122000CE08FC01EE0FFF1FE85FFE4F20813181E9
:10123000232B39F421E030E03183208361E00C94EA
:101240005D030895CF93C82F0E940B09CE3018F08C
:1012500082EF8C0F01C08C2F8770806480937C009C
:1012600080917A00806480937A0080917A0086FD74
:10127000FCCF609178008091790070E0782B072E88
:10128000000C880B990B0E942D140E94D3088C2F00
:101290000E94CE0882E00E94CE08CF910C94FB08F9
:1012A0003FB7F8948091880390918903A0918A03B5
:1012B000B0918B0326B5A89B05C02F3F19F001966E
:1012C000A11DB11D3FBFBA2FA92F982F8827820FCC
:1012D000911DA11DB11DBC01CD0142E0660F771F1C
:1012E000881F991F4A95D1F708951F920F920FB644
:1012F0000F9211242F933F938F939F93AF93BF939C
:101300008091840390918503A0918603B091870317
:101310003091830323E0230F2D3720F40196A11D84
:10132000B11D05C026E8230F0296A11DB11D209313
:1013300083038093840390938503A0938603B093E3
:1013400087038091880390918903A0918A03B091CB
:101350008B030196A11DB11D80938803909389038F
:10136000A0938A03B0938B03BF91AF919F918F910C
:101370003F912F910F900FBE0F901F901895CF9215
:10138000DF92EF92FF920F931F93E82FF92F05C082
:10139000015011092109310961F1908196239417B7
:1013A000B9F305C0015011092109310911F19081EA
:1013B00096239413F7CFC12CD12CE12CF12C0AC029
:1013C0008FEFC81AD80AE80AF80A0C151D052E0571
:1013D0003F0579F080818623841791F36C2D7D2D54
:1013E0008E2D9F2D1F910F91FF90EF90DF90CF904A
:1013F000089560E070E080E090E01F910F91FF9011
:10140000EF90DF90CF900895CF93DF9300D000D07E
:1014100000D0CDB7DEB7789484B5826084BD84B542
:10142000816084BD85B5826085BD85B5816085BDDF
:1014300080916E00816080936E0010928100809197
:10144000810082608093810080918100816080931F
:101450008100809180008160809380008091B10044
:1014600084608093B1008091B00081608093B0006F
:1014700080917A00846080937A0080917A00826003
:1014800080937A0080917A00816080937A008091C5
:101490007A00806880937A001092C10060E08EE04C
:1014A0000E945D0360E08FE00E945D0362E082E0E5
:1014B0000E945D0362E087E00E945D0361E084E0DA
:1014C0000E945D0360E084E00E94DA0261E081E155
:1014D0000E945D0361E081E10E94DA0261E080E147
:1014E0000E945D0361E080E10E94DA0261E081E137
:1014F0000E945D0361E081E10E94DA0261E080E127
:101500000E945D0361E080E10E94DA0261E083E015
:101510000E945D0360E083E00E94DA0261E085E002
:101520000E945D0360E085E00E94DA0261E086E0EF
:101530000E945D0360E086E00E94DA0261E089E0DB
:101540000E945D0360E089E00E94DA0261E08AE0C7
:101550000E945D0360E08AE00E94DA0261E08BE0B5
:101560000E945D0361E08BE00E94DA0261E08CE0A2
:101570000E945D0361E08CE00E94DA0261E08DE090
:101580000E945D0361E08DE00E94DA020E9409037F
:1015900080E20E94FE018FEF90E00E949C000E947A
:1015A000A20181E20E94FE018FEF90E00E949C0068
:1015B0000E94A20182E20E94FE018FEF90E00E9451
:1015C0009C000E94A20183E20E94FE018FEF90E046
:1015D0000E949C000E94A20184E20E94FE018FEF03
:1015E00090E00E949C000E94A20185E20E94FE0100
:1015F0008FEF90E00E949C000E94A20186E20E9470
:10160000FE018FEF90E00E949C000E94A20187E201
:101610000E94FE018FEF90E00E949C000E94A201B8
:101620000E943B0310921D0310921E0310921F0391
:10163000109220030E94080280910C0390910D03E8
:1016400097FD08C061E00E945D0360E080910C039B
:101650000E94DA0281E08093070380910803909151
:101660000903892B01F1209114033091110380911A
:101670000F0390911003231721F0FC01E20FF11DDD
:10168000108220911103FC01E20FF11D10822091C4
:101690001203FC01E20FF11D108220911303FC01E3
:1016A000E20FF11D10828AE00E9461010E94A100F8
:1016B000E0914802F091490282E08083E091480283
:1016C000F09149021082E0914402F09145021082AB
:1016D000E0914602F091470280E18083109250022F
:1016E000E0914C02F0914D0286E08083E0914A0245
:1016F000F0914B02808180618083E0914A02F091F9
:101700004B02808188608083E0914A02F0914B0215
:10171000808180688083E0914A02F0914B02808151
:101720008F7D808361E2262E63E0362E88E392E08F
:101730000E948D04892B09F452C488E392E00E9430
:101740008D041816190694F788E392E00E946B0442
:101750009091BE01853561F491110AC08091BD015F
:101760008F3FE1F481E08093BC018093BE0116C0FD
:101770008093BD01992391F0E091BC01E23019F40E
:101780008093BB0107C0E33028F09091BB019150DA
:101790009093BB01F0E0E957FE4F80838091BC013C
:1017A0008F5F843318F48093BC0104C01092BC0195
:1017B0001092BE018091BE01882309F4B7CF8091B9
:1017C000BB018111B3CF8091BC01843008F4AECF4E
:1017D0001092BE0100918B01E0918C01D0908D019F
:1017E000ED2CF12CF0928601E092850110918E0192
:1017F000212F30E03A832983023009F48BC0033073
:1018000009F4E8C3013009F0E7C3E73009F058C034
:101810008091C601811119C00093C601F0920401A4
:10182000E09203013093020120930101F701EE0FD2
:10183000FF1FE85FFE4F81E090E091838083220FDD
:10184000331F285F3E4FF9012AC080910301909118
:101850000401E816F90651F480910101909102010A
:1018600029813A812817390709F4B6C3F092040197
:10187000E092030189819A81909302018093010192
:10188000F701EE0FFF1FE85FFE4F81E090E09183CC
:101890008083E981FA81EE0FFF1FE85FFE4F91839D
:1018A000808361E08D2D0E945D0362E0812F0E94A4
:1018B0005D0362E370E080E090E00E94F8038CC377
:1018C000EC3039F400930701F0920601E092050133
:1018D00083C32091030130910401C701880F991F30
:1018E000E216F30639F02091010130910201E2166F
:1018F000F30651F41092C6011092C1011092C20178
:101900001092C3011092C401FC01E85FFE4F1182E6
:10191000108262C32091030130910401E216F306A4
:1019200039F02091010130910201E216F30651F4E1
:101930001092C6011092C1011092C2011092C3010F
:101940001092C4018E2FEE0F990BAA0BBB0BFC015A
:101950003197EE30F10508F03DC3EC5CFF4F0C947D
:101960006315C7010E941109612F8D2D0E94DA02B3
:1019700031C3C7010E9411091093690180918F0141
:1019800080936A012091690130916A013E832D8321
:1019900080919001809369018091910180936A0107
:1019A0008091690190916A019A83898318161906BA
:1019B0000CF0ACC180910001D81621F08F3F09F0E6
:1019C00009C304C0E4E8F0E0049174C0D0920001BF
:1019D000E4E8F0E0E491EF3F09F4FCC2E13009F4FF
:1019E00043C038F1E23009F064C01092B0001092A8
:1019F000B1008091B00082608093B0008091B1000E
:101A000081608093B100F701E553FF4FE491F0E06E
:101A1000EE0FFF1FEF53FF4F85919491909360015C
:101A200080935F01F701E355FF4FE491E0935E017E
:101A300000C514BC15BC84B5826084BD85B58160C9
:101A400085BDF701E553FF4FE491F0E0EE0FFF1F76
:101A5000EF53FF4F85919491F701E355FF4FE491C8
:101A6000E0936C0100E0E5C41092800010928100C8
:101A700080918100886080938100809181008160E5
:101A800080938100F701E553FF4FE491F0E0EE0F02
:101A9000FF1FEF53FF4F85919491F701E355FF4FDF
:101AA000E491E0936B0161E08D2D0E945D0301E004
:101AB000B4C00E2F07FD8EC261E08D2D0E945D0324
:101AC000802F8D7F09F0A9C0ED81FE814F01A12CEF
:101AD000B12C60E072E18AE790E0A50194010E94D8
:101AE0002E1329013A0169017A01F1E0CF1AD108D8
:101AF000E108F1082FEFC216D104E104F10409F066
:101B000008F44BC060E472E48FE090E0A50194011A
:101B10000E942E1369017A0181E0C81AD108E108F8
:101B2000F108023001F59FEFC916D104E104F10478
:101B300009F008F416C460E970ED83E090E0A501B7
:101B400094010E942E1369017A01E1E0CE1AD108B6
:101B5000E108F108FFEFCF16D104E104F10409F028
:101B600030F583E053C02FEFC216D104E104F10435
:101B7000B1F0A8F068E478EE81E090E0A50194016E
:101B80000E942E1369017A0181E0C81AD108E10888
:101B9000F108002309F41AC410C481E001C082E0F6
:101BA000011134C095B5987F892B85BD6AC068E462
:101BB00078EE81E090E0A50194010E942E13690166
:101BC0007A01F1E0CF1AD108E108F1082FEFC2162F
:101BD000D104E104F10409F008F4C1C364E274EF34
:101BE00080E090E0A50194010E942E1369017A0122
:101BF00091E0C91AD108E108F108EFEFCE16D1043F
:101C0000E104F10411F008F0AEC385E09091B10059
:101C1000987F892B8093B10034C02D813E8149018A
:101C2000A12CB12C60E072E18AE790E0A50194015B
:101C30000E942E1369017A0181E0C81AD108E108D7
:101C4000F108C114D10491E0E906F10488F068E4D8
:101C500078EE81E090E0A50194010E942E136901C5
:101C60007A01E1E0CE1AD108E108F10883E001C071
:101C700081E0013031F490918100987F892B80932D
:101C800081002D813E81220F331FA981BA810E94DC
:101C9000691528EE33E040E050E00E944D1301301A
:101CA00099F0023019F1011195C1C7BC209371015F
:101CB00030937201409373015093740180916E00D0
:101CC000826080936E0086C1D0928900C0928800A5
:101CD00020936D0130936E0140936F01509370011A
:101CE00080916F00826080936F0074C1C092B300D6
:101CF000209361013093620140936301509364012A
:101D00008091700082608093700064C18D2D0E946C
:101D1000000660C1C7010E941109153B08F05AC1B5
:101D2000E5E7F1E080E090E021913191E216F306E1
:101D300081F0232B41F4FC01EE0FFF1FEB58FE4F07
:101D4000F182E08206C001968830910569F780E053
:101D500090E09C01220F331F820F931FFC01ED5D69
:101D6000FC4F00810C3008F035C161E08D2D0E94E0
:101D70005D0310E0C801880F991FFC01E00FF11FFF
:101D8000EF51FD4F2D2D2F733081307CD32ED22A71
:101D9000D08220E030E0F901EE0FFF1FE20FF31FC9
:101DA000EF51FD4F408146FD14C02F5F3F4F2C3057
:101DB000310589F71092800022E020938100109273
:101DC000850010928400B19A20916F0022602093C8
:101DD0006F00800F911FFC01EF51FD4F80818064E7
:101DE0008083A981BA81A53BB10514F0A4EBB0E0D2
:101DF00020E437E00E94691524EB30E040E050E039
:101E00000E942E13DA01C901805E9D4FAF4FBF4F74
:101E10009C018136994014F020E639E022503109C6
:101E2000220F331F8FB7F894F801EE0FFF1F0E0F2C
:101E30001F1FF801EF51FD4F328321838FBFCAC0AE
:101E400000919001202F30E03A83298361E085E002
:101E50000E945D0361E086E00E945D03011105C000
:101E60001092C00160E070E00DC081E08093C0017D
:101E7000111102C061E001C060E085E00E94DA0259
:101E800069817A8186E023C000919001802F90E0E3
:101E90009A83898361E089E00E945D0361E08AE0C2
:101EA0000E945D03011105C01092BF0160E070E067
:101EB0000DC081E08093BF01111102C061E001C03B
:101EC00060E089E00E94DA0269817A818AE00E94FA
:101ED000990380C090E2E91AF108E8E0EE16F104F7
:101EE00050F48D2D0E94FE0189819A810E949C00F0
:101EF0000E94A2016FC0D1106DC00E943B031093DD
:101F0000650180918F01809366018091900180939B
:101F100067018091910180936801609165017091E2
:101F2000660180916701909168010E94F5136D83AD
:101F3000798380E090E00E942B1420E03CE34CE1A8
:101F400056E40E94DD14EDE1F3E01816FCF028EEF3
:101F500033E08D819981B9010E944F15DB01A45DA9
:101F6000BE4F4C91542F5F7740814078452B419371
:101F70008D839983C9016AE070E00E944F159B012F
:101F80002E163F0631F70E94080224C08081807817
:101F90008F6681932E163F06C9F7F5CF0091900109
:101FA000F0918F01FD83402F6F2F812F0E94380207
:101FB000209191012983822F0E9461010E94A1003A
:101FC000402F6D81812F0E94380289810E9461011A
:101FD0000E94A1000E9403091092BC01A7CB6FE0F0
:101FE00070E080E090E00E94F80368E0E62E61E097
:101FF000F62E1A821982F701019111917F010115C4
:10200000110509F051C08091C001882331F0898108
:102010009A810597029708F445C08091BF018823F3
:1020200031F089819A810997029708F43BC0B98001
:1020300062E08B2D0E945D030E940B09E981FA8109
:10204000E756FF4F8491E981FA81E355FF4FC49031
:10205000E981FA81E553FF4FD490DD2099F0811199
:102060000E94B102ED2DF0E0EE0FFF1FEB57FF4F86
:10207000A591B491EC91CE2291E080E009F490E03A
:10208000092F182FB801110F880B990B0E942D14DE
:102090000E94D3088B2D0E94CE0881E00E94CE08BA
:1020A0000E94FB080E94030929813A812F5F3F4F5C
:1020B0003A8329832E30310509F09DCF80E090E0EE
:1020C0000E9422090E94030981E090E00E942209F7
:1020D0000E94030987E090E00E9422090E94030900
:1020E0008091C701803108F44AC01092C7010E9454
:1020F0000B0980911C030E94FE0180E090E00E9489
:102100009C000E94A20162E080911C030E946F0269
:102110001092370280933602811103C06FEF7FEF78
:1021200015C085ED92E00E94820589839091360268
:1021300080913702981791F385ED92E00E94820515
:1021400039813C831B826B817C81682B072E000CBC
:10215000880B990B0E942D1420E030E040E85BE3EF
:102160000E94E2140E94D30880E00E94CE088FE013
:102170000E94CE080E94FB080E94030903C08F5FE3
:102180008093C7018091C601882309F496C080918D
:102190000301898360E00E94DA0283E090E0019706
:1021A000F1F761E089810E94DA0283E290E0019711
:1021B000F1F760E089810E94DA028091010190913B
:1021C00002019927FC01E355FF4F6491FC01E5539F
:1021D000FF4FE491F0E0EE0FFF1FEB57FF4F8591AB
:1021E000949100E315E720E030E0462F0E94BF09FC
:1021F000611571058105910549F0DC01CB0101965E
:10220000A11DB11DBC01CD019F7003C060E070E055
:10221000CB010E942B1420E030E048EE51E40E94F4
:10222000831320E030E040E05FE30E94E2146B01A2
:102230007C0120E030E0A9010E947E1381111EC0C4
:102240008091C501853670F01092C6011092C101CF
:102250001092C2011092C3011092C401C12CD12C62
:10226000760116C08F5F8093C501C090C101D090E8
:10227000C201E090C301F090C4010AC0C092C10144
:10228000D092C201E092C301F092C4011092C50144
:102290000E940B09C701B6010E94D3088091030177
:1022A0000E94CE08809101010E94CE0887E00E9422
:1022B000CE080E94FB080E94030980910701882331
:1022C00009F440C0E0910501F0910601FA83E98329
:1022D000CF0180970897B0F561E089810E946F0275
:1022E00010923702809336026AE070E080E090E05E
:1022F0000E94F8038091360290E020913702821B01
:1023000091090197F9F485ED92E00E9482058D8391
:102310000E940B0984E00E94CE0880E00E94CE0853
:1023200080E00E94CE0880E00E94CE088D818095DA
:102330000E94CE0889810E94CE088CE00E94CE08BF
:102340000E94FB0888E392E00E9412056AE070E0B8
:1023500080E090E00E94F8030E943405E3C984E025
:1023600055CC82E053CC62E17AE780E090E0A501B1
:1023700094010E942E1369017A01F1E0CF1AD1086D
:10238000E108F1088FEFC816D104E104F10499F0D7
:1023900090F0D301C2013AE0B595A795979587953E
:1023A0003A95D1F76C017D0131E0C31AD108E108FB
:1023B000F10887E02BCC86E029CC2FEFC216D104A0
:1023C000E104F10409F078F684E0EACBEFEFCE16F1
:1023D000D104E104F10459F150F162E17AE780E0BF
:1023E00090E0A50194010E942E1369017A0181E019
:1023F000C81AD108E108F1089FEFC916D104E10419
:10240000F10499F090F0D301C2012AE0B595A795A7
:10241000979587952A95D1F76C017D01E1E0CE1A59
:10242000D108E108F10885E0BDCB84E0BBCB83E0B7
:10243000B9CB61E08D2D0E945D0346CB10923B022B
:1024400010923A0288EE93E0A0E0B0E080933C0264
:1024500090933D02A0933E02B0933F022AE331E005
:10246000309339022093380225EC30E03093450256
:102470002093440224EC30E030934702209346023C
:1024800020EC30E0309349022093480221EC30E008
:1024900030934B0220934A0222EC30E030934D02FD
:1024A00020934C0226EC30E030934F0220934E02F2
:1024B0001092510210925202109253021092540242
:1024C0001092D8021092D7028093D9029093DA0228
:1024D000A093DB02B093DC028CE491E09093D602EF
:1024E0008093D50280910503A3E2B3E09FEF48EB10
:1024F0005BE08C3078F48C93282F30E0F901EE0FFC
:10250000FF1F2E0F3F1FF901EF51FD4F52834183F3
:102510008F5F01C09C93139623E0AB33B20749F75A
:10252000809305038C30A0F491E0980F90930503FD
:1025300080933C0390E0FC01EE0FFF1F8E0F9F1F66
:10254000FC01EF51FD4F88EB9BE09283818303C038
:102550008FEF80933C0380E790E090932203809379
:10256000210310921D0310921E0310921F0310925C
:1025700020030E94090388E480931C031092070340
:1025800010920E0310921503109216031092170367
:102590001092180381E0809314038093110310922A
:1025A000120392E0909313038093060383E090E07C
:1025B00090930B0380930A030E947015909310036D
:1025C00080930F03009761F023E0FC0111922A959C
:1025D000E9F781E090E0909309038093080308C035
:1025E00010920B0310920A03109209031092080331
:1025F00088E090E090930D0380930C038091070393
:10260000882341F061E088E00E945D0360E088E09B
:102610000E94DA02E3EDF0E0E491F0E0EE0FFF1F3C
:10262000EF53FF4F8591949190931A038093190370
:10263000E5EBF0E0E491E0931B03089580910F0334
:10264000909110030E94081680910C0390910D0345
:1026500097FD03C060E00C945D030895052E97FB81
:102660001EF400940E94451357FD07D00E944D139D
:1026700007FC03D04EF40C944513509540953095CB
:1026800021953F4F4F4F5F4F0895909580957095DE
:1026900061957F4F8F4F9F4F0895A1E21A2EAA1B7D
:1026A000BB1BFD010DC0AA1FBB1FEE1FFF1FA21702
:1026B000B307E407F50720F0A21BB30BE40BF50BFF
:1026C000661F771F881F991F1A9469F76095709588
:1026D000809590959B01AC01BD01CF010895A29F0B
:1026E000B001B39FC001A39F700D811D1124911DE6
:1026F000B29F700D811D1124911D08950E946814D0
:1027000008F481E008950E9497130C94A3140E948A
:102710009C1458F00E94951440F029F45F3F29F072
:102720000C948C1451110C94D7140C9492140E9494
:10273000B41468F39923B1F3552391F3951B550B0A
:10274000BB27AA2762177307840738F09F5F5F4F84
:10275000220F331F441FAA1FA9F335D00E2E3AF0C3
:10276000E0E832D091505040E695001CCAF72BD0DB
:10277000FE2F29D0660F771F881FBB1F261737072C
:102780004807AB07B0E809F0BB0B802DBF01FF275E
:1027900093585F4F3AF09E3F510578F00C948C149B
:1027A0000C94D7145F3FE4F3983ED4F38695779565
:1027B0006795B795F7959F5FC9F7880F911D969517
:1027C000879597F90895E1E0660F771F881FBB1F73
:1027D000621773078407BA0720F0621B730B840B20
:1027E000BA0BEE1F88F7E09508950E94FC136894D9
:1027F000B1110C94D71408950E94BC1488F09F570F
:1028000098F0B92F9927B751B0F0E1F0660F771F14
:10281000881F991F1AF0BA95C9F714C0B13091F00A
:102820000E94D614B1E008950C94D614672F782F27
:102830008827B85F39F0B93FCCF3869577956795CF
:10284000B395D9F73EF490958095709561957F4F3B
:102850008F4F9F4F0895E89409C097FB3EF49095E1
:102860008095709561957F4F8F4F9F4F9923A9F069
:10287000F92F96E9BB279395F695879577956795F8
:10288000B795F111F8CFFAF4BB0F11F460FF1BC03C
:102890006F5F7F4F8F4F9F4F16C0882311F096E9CF
:1028A00011C0772321F09EE8872F762F05C066237D
:1028B00071F096E8862F70E060E02AF09A95660F36
:1028C000771F881FDAF7880F9695879597F90895EF
:1028D000990F0008550FAA0BE0E8FEEF1616170631
:1028E000E807F907C0F012161306E407F50798F099
:1028F000621B730B840B950B39F40A2661F0232BB2
:10290000242B252B21F408950A2609F4A140A6952D
:102910008FEF811D811D089597F99F6780E870E012
:1029200060E008959FEF80EC089500240A94161645
:10293000170618060906089500240A9412161306AD
:10294000140605060895092E0394000C11F488233B
:1029500052F0BB0F40F4BF2B11F460FF04C06F5F57
:102960007F4F8F4F9F4F089557FD9058440F551F2D
:1029700059F05F3F71F04795880F97FB991F61F001
:102980009F3F79F087950895121613061406551F78
:10299000F2CF4695F1DF08C0161617061806991FE4
:1029A000F1CF86957105610508940895E894BB27D9
:1029B00066277727CB0197F908950E94681408F4D9
:1029C0008FEF08950E94F5140C94A3140E9495149F
:1029D00038F00E949C1420F0952311F00C948C1474
:1029E0000C94921411240C94D7140E94B41470F314
:1029F000959FC1F3950F50E0551F629FF001729FA4
:102A0000BB27F00DB11D639FAA27F00DB11DAA1FB2
:102A1000649F6627B00DA11D661F829F2227B00DFF
:102A2000A11D621F739FB00DA11D621F839FA00D8A
:102A3000611D221F749F3327A00D611D231F849FDA
:102A4000600D211D822F762F6A2F11249F57504031
:102A50009AF0F1F088234AF0EE0FFF1FBB1F661FAC
:102A6000771F881F91505040A9F79E3F510580F075
:102A70000C948C140C94D7145F3FE4F3983ED4F379
:102A8000869577956795B795F795E7959F5FC1F719
:102A9000FE2B880F911D9695879597F90895AA1B8F
:102AA000BB1B51E107C0AA1FBB1FA617B70710F039
:102AB000A61BB70B881F991F5A95A9F7809590956B
:102AC000BC01CD010895EE0FFF1F0590F491E02D9C
:102AD00009940E946F13B7FF0895821B930B08950A
:102AE0000F931F93CF93DF938230910510F482E010
:102AF00090E0E0918E03F0918F0320E030E0A0E0C1
:102B0000B0E0309719F1408151810281138148175B
:102B10005907C8F08417950769F4109731F0129699
:102B20000C93129713961C9327C000938E03109357
:102B30008F0322C02115310519F04217530718F4ED
:102B40009A01BD01EF01DF01F801DBCF211531054D
:102B5000F9F0281B390B2430310580F48A819B81E0
:102B60006115710521F0FB019383828304C090936A
:102B70008F0380938E03FE01329644C0FE01E20F64
:102B8000F31F8193919322503109398328833AC0EE
:102B900020918C0330918D03232B41F42091280147
:102BA0003091290130938D0320938C0320912601CD
:102BB000309127012115310541F42DB73EB74091E1
:102BC0002A0150912B01241B350BE0918C03F091CD
:102BD0008D03E217F307A0F42E1B3F0B28173907CC
:102BE00078F0AC014E5F5F4F2417350748F04E0F69
:102BF0005F1F50938D0340938C038193919302C088
:102C0000E0E0F0E0CF01DF91CF911F910F910895A7
:102C1000CF93DF93009709F481C0FC0132971382B0
:102C20001282A0918E03B0918F03109781F42081BE
:102C30003181820F931F20918C0330918D032817CF
:102C4000390751F5F0938D03E0938C0367C0ED01D4
:102C500020E030E0CE17DF0740F44A815B819E011F
:102C600041155105F1F0EA01F5CFD383C2834081CC
:102C70005181840F951FC817D90759F4888199810C
:102C8000840F951F0296918380838A819B81938311
:102C900082832115310529F4F0938F03E0938E038D
:102CA0003DC0E901FB83EA8349915991C40FD51FC7
:102CB000EC17FD0761F480819181840F951F0296C6
:102CC000E90199838883828193819B838A83E0E0F1
:102CD000F0E012968D919C911397009719F0FD01E9
:102CE000DC01F7CF8D919C9111979D012E5F3F4F95
:102CF000820F931F20918C0330918D032817390781
:102D000069F4309729F410928F0310928E0302C059
:102D100013821282B0938D03A0938C03DF91CF9125
:102D2000089581E090E0F8940C94961610E0C1E7C5
:102D3000D0E004C0FE010E9463152196C237D1077E
:062D4000C9F7F894FFCF73
:102D4600FF0C000D0027000100000000000000003D
:102D56000100000001000000010000000100000069
:102D66000000000000000000900380003F065B4F5B
:102D7600666D7D077F6F00000000C50432045C04A9
:102D860012058D046B047F0400000000CB059E0530
:0E2D9600FB0572059605820573050D0A000007
:00000001FF
